:02000000AE2B25
:020008000029CD
:02000E00820767
:10001000443453344334203432342E343034303486
:10002000323432342F34303433342F3430343834A3
:100030004E346534783474342034533465346C343D
:100040005234653476342034443465346334203497
:10005000523465347634203452342F3441342034D1
:100060002034423472346934673468347434203450
:1000700043346F346E347434723461347334743492
:10008000533479347334523465347334653474348E
:10009000443465346634613475346C347434733488
:1000A00045347834693474344D3465346E34753481
:1000B0005234653476342034203453346534743407
:1000C000523465347634443420344F3466346634E4
:1000D000523465347634443420344F346E34203412
:1000E000523465347634523420344F3466346634B6
:1000F000523465347634523420344F346E342034E4
:1001000049346E34633420342034533465347434C9
:10011000423472346934673468347434203420349F
:1001200043346F346E34743420342034203420341B
:10013000593465347334203420344E346F342034D1
:100140002034523465347334653474343F3420348D
:10015000443465346634613475346C3474343F34FB
:1001600046346F346334753473344F3475347434B7
:1001700046346F34633475347334203449346E3408
:10020000A600030EA7000B1930298B182029270EF2
:100210008300A60E260E09006400810183160313D5
:1002200088308100831286140614A50183160313F7
:1002300019309900243098008312903098000800FB
:100240008B100C30A000A00B232906180729AD3015
:10025000810020308B000230A5000830A000072963
:100260000B1125194329A00803193C29060CA10CE0
:10027000A003AD3081000729061C59290130A500D3
:100280002108A2005929A5195929A00803195129A3
:10029000A30C031C861003188614A003B53081003C
:1002A00007290000000000008614A515A830810071
:1002B000072900308B000130A50507296400A80B31
:1002C0006E29A90B772C0130AA06031D6929071492
:1002D0006A2907100030A8001830A9003030050541
:1002E000B1003202031D7F210C300505B9003A022E
:1002F000031DA9213108B2003908BA0008003208EC
:100300003106303C0319D329310DB206B21E9929AA
:1003100041189B29AD08031D9729AE08031D962996
:100320002B08AD002C08AE00AD080319AE03AD03D9
:10033000080041188A29AD0A0319AE0A2B082D02BC
:10034000031D08002C082E02031D0800AD01AE019C
:1003500008003A0839060C3C0319D329390DBA06AE
:10036000BA1DC3294218C529B508031DC129B608FD
:10037000031DC0293308B5003408B600B5080319B9
:10038000B603B50308004218B429B50A0319B60A22
:1003900033083502031D080034083602031D080027
:1003A000B501B6010800BB0A080087145E218C1E47
:1003B000D6299818E129181DE329181218161A08C9
:1003C0000800181218161A08A20087100800A300C7
:1003D0005E210C1EE8292308990007115E210C1EDE
:1003E000EE2907150800633084001030DC00D521A9
:1003F00022088000840ADC0BF7295708013C031D02
:10040000182AC308031D182A42220830DC00633072
:100410008400640000083022840ADC0B092A5A2276
:100420000830DC00640000083022840ADC0B122A49
:100430000F24FD2B1C22242ADB000830DB02422281
:10044000252ADB000830DB025A220830DC000030AD
:100450008A005B0807203022DB0ADC0B272A080011
:10046000A3005E21A518312A86100630A5000000E1
:10047000B5308100A0308B000830A0005E21A518A7
:100480003E2A0800FE3030224830302AFE3030222A
:10049000993030225E08522AFE303022503030220D
:1004A0005F08522A0310DA00DA0DDA0DDA07DA0DE6
:1004B0005A0D302AFE3030224730302201303022AF
:1004C0000230302AFE3030224730302208303022CD
:1004D0000130302ACE223F08B3003E08B400CE22BD
:1004E0003F08AB003E08AC0079225230E7210F24D0
:1004F000FD2B8312031700308D002B088C00B122D6
:100500008312031701308D002C088C00B122831256
:10051000031702308D0033088C00B12283120317B9
:1005200003308D0034088C00B12A83120317043085
:100530008D0041088C00B12A8312031705308D000D
:1005400042088C00B12A8312031706308D005E0822
:100550008C00B12A8312031707308D005F088C00CE
:10056000B12A6400831603130D16831203130D12B0
:100570008B130B17831603178C130C1555308D0036
:10058000AA308D008C1463000C11831603130D1216
:10059000831203130D120B138B17080063308400B2
:1005A000A401BF01BE01A408031DE42AD52122082D
:1005B000203C0319D32A22080D3C0319D32A220810
:1005C0008000A40A840AD62A84030030BC000130CB
:1005D000BD000E23A40BED2A080084030030BC00EC
:1005E0000A30BD000E23A40BF62A08008403003055
:1005F000BC006430BD000E23A40BFF2A0800840356
:100600000330BC00E830BD000E23A40B082B08000B
:1006100084032730BC001030BD000E2B2F300002A9
:10062000C000C00B142B08003D08BF070318BE0A0A
:100630003C08BE07112B3B08BD00BC018B232030BA
:10064000E7214108303EE7212030E7214208303ED3
:10065000E7212030E7210508BD00BC018B230F24D2
:10066000BB01FD2B2D08AF002E08B0003508B700E8
:100670003608B8003708BD003808BC0048230930E8
:10068000E7212F08BD003008BC0048230F24FD2BB4
:100690002B30E7217D2BCE223F08C100952244302C
:1006A000E7213F08303EE7210F24FD2BCE223F08F3
:1006B000C2009C225230E7213F08303EE7210F2440
:1006C000FD2BCE223F08B5003E08B600CE223F08E3
:1006D000AD003E08AE005330E7210F24FD2B340857
:1006E000BC003308BD007D232030E7212C08BC006E
:1006F0002B08BD007D230F24FD2B2730BE001030BA
:10070000BF009C234008E7210330BE00E830BF0053
:100710009C234008E7210030BE006430BF009C23CA
:100720004008E7210030BE000A30BF009C2340088B
:10073000E7213D08303EE7292F30C000C00A3F08BE
:10074000BD023E08031C013EBC0203189E2B3F085D
:10075000BD073E080318013EBC07080083120313BF
:100760008501831606309F00FF308500FD3086002E
:10077000C030870083120313071207140030AA0049
:10078000A8001830A9008714071587158712303084
:100790000505B2000C300505BA00C501C3010830DB
:1007A000C8000130C6000C21132400308B00FF303C
:1007B000D000CF00CE00CD00CC00CB00CA00C900D5
:1007C000D100D500D400D300D200D6000130D7002C
:1007D0000030D800D900C8309525C830952546226C
:1007E0004C221630DC0007308A005C08163CC0271B
:1007F0003022DC0BF32B08301A22D52107308A0077
:10080000DA015A08D727FF390319FD2B22020319F1
:100810000B2CDA0A012C07308A005A08E12F0D3020
:10082000E7210A30E72964008312031700308D00A6
:10083000831603178C130C14831203170C08AB00D8
:1008400001308D00831603178C130C1483120317C9
:100850000C08AC0002308D00831603178C130C14A7
:10086000831203170C08B30003308D00831603179F
:100870008C130C14831203170C08B40004308D0081
:10088000831603178C130C14831203170C08C10072
:1008900005308D00831603178C130C148312031775
:1008A0000C08C20006308D00831603178C130C143D
:1008B000831203170C08DE0007308D008316031720
:1008C0008C130C14831203170C08DF000313BB01F5
:1008D0003308B5003408B6000310B60CB50C2B086D
:1008E000AD002C08AE000310AE0CAD0C0800640087
:1008F0004F08D0004E08CF004D08CE004C08CD0068
:100900004B08CC004A08CB004908CA000608C03989
:10091000C90050084F044E044D044C044B044A04D3
:100920004904D100C0390319E02C5708013C031DCC
:10093000F12C3230C4005108C03C0319BD2C5208C0
:10094000530454045504DA00DA1FD92C5A1FD32C4F
:1009500048080319AD2CC803CF2C5408D500530800
:10096000D4005208D3005108D2004030C8000130F2
:10097000C400D11FD62C511FD02CFF30D000CF0087
:10098000CE00CD00CC00CB00CA00C900D100D500FC
:10099000D400D300D2000830C8000030C5006E2952
:1009A000C308031DCF2C0230C600DB2CC308031D77
:1009B000CF2C0130C6004408C5000130C300CF2C45
:1009C00064005708023C0319CF2C0230D7000030D6
:1009D000D800D9001830212220301C225108D6001E
:1009E000CF2C6400560851020319CF2CD608031DE2
:1009F000002D5108C03A031DCF2C5108D600CF2C32
:100A00005108D600511F2D2DD11F072DBD2C580880
:100A1000013C0319822D0130D80007308A005908A3
:100A2000EA2F640058302122372D640058302122EB
:100A30003F2D6400803021224A2D64008030212225
:100A4000582D640098302122A0301C22CF2C640045
:100A500098302122A8301C22CF2C580803197C2D55
:100A600007308A005908F22F0130C1069522603004
:100A7000411868301C22CF2C0130C2069C227030F5
:100A8000421878301C22CF2C5E080A3C0319DE0184
:100A9000DE0AA32288301C2262225E082F3E30220A
:100AA0004622CF2C5F080A3C0319DF01DF0AAA2285
:100AB00090301C2262225F082F3E30224C22CF2C25
:100AC000AE2B0301AB00B3002030AC00B4007922A0
:100AD0000301C100C20095229C220630DE00DF0027
:100AE000A322AA2246224C22822D0030D8000130B7
:100AF000D70008301A22CF2C5908013ED900073CF4
:100B00000319D9010310D8015908DA00DA0DDA0DFA
:100B1000DA0D20305A071C2218302122CF2C7C30CD
:100B2000E1006400E10B912D0800E2008F25E20B4B
:040B3000962D0800F6
:100F80008207FE344E34013404340E3415340434F4
:100F90000434043404340034FE344E340234043453
:100FA00004340434043415340E3404340034820719
:100FB00051345634763453345234483471344C34CA
:100FC00000348207322B4B2B562B612B6A2A6F2B56
:100FD0001B2BF3298207112D152D192D1D2D212DC8
:100FE000272D752D8207342D3C2D442D522D602D3B
:040FF000612D752DCD
:02400E00713F00
:104200000000200000002000000000000600060062
:00000001FF
